:020000040800F2
:10000000A0080020010100084D0D0008B70C0008F1
:100010004B0D0008DD020008051A00080000000072
:100020000000000000000000000000006110000857
:10003000A509000800000000350F0008651600083B
:100040001B0100081B0100081B0100081B01000820
:100050001B0100081B0100081B0100081B01000810
:100060001B0100081B0100081B010008990400087F
:100070001B0100081B0100081B0100081B010008F0
:100080001B0100081B0100081B0100081B010008E0
:10009000951900081B0100081B0100081B0100083E
:1000A0001B0100081B0100081B010008B91600080D
:1000B0001B0100081B0100081B0100081B010008B0
:1000C0001B0100081B0100081B0100081B010008A0
:1000D0001B0100081B0100081B0100081B01000890
:1000E0001B0100081B0100081B010008DFF80CD0F1
:1000F00000F018F800480047B11C0008A0080020D4
:100100000648804706480047FEE7FEE7FEE7FEE7B1
:10011000FEE7FEE7FEE7FEE7FEE7FEE769160008FA
:10012000ED000008064C074D06E0E06840F00103D2
:1001300094E8070098471034AC42F6D3FFF7DAFF93
:10014000A01D0008C01D00080029816802D041F0F0
:10015000010101E021F001018160704710B54FF409
:10016000004000F021FF16480021164C016001718B
:1001700041718160C160012101740146204600F097
:1001800045F8012205231146204600F063F80121BD
:10019000204600F019F801212046FFF7D5FF204640
:1001A00000F092F8204600F02AF80028FAD1204604
:1001B00000F08FF8204600F01BF80028FAD110BD9F
:1001C000C4030020002401400029816802D041F4CA
:1001D000807101E021F4807181607047002981689D
:1001E00002D041F4801101E021F480118160704758
:1001F000014600208968490700D501207047014663
:1002000000208968090700D50120704710B54268B1
:100210000E4B0C791A400B6842EA042213434360E8
:1002200083680B4A1340D1E9024222434C7943EAE6
:1002300044031A438260C26A097C22F47002491E98
:10024000C9B242EA0151C16210BD0000FFFEF0FFD9
:10025000FDF7F1FF70B5072509290AD9C468A1F196
:100260000A0606EB4606B540AC43B3401C43C460E7
:1002700007E0046901EB4106B540AC43B3401C43C1
:1002800004611F23072A09D2446B521E02EB82022B
:1002900093409C4391400C43446370BD0D2A09D2A6
:1002A000046BD21F02EB820293409C4391400C43AB
:1002B000046370BDC46A0D3A02EB820293409C4312
:1002C00091400C43C46270BD816841F008018160B7
:1002D0007047816841F0040181607047FEE7C1B258
:1002E000000A40EA012070472DE9F84FDFF82CA101
:1002F0004BF6BF7648F28007474D40F68F78474C63
:1003000048F60F7BDFF818910AF1440A2CE00188C7
:1003100011F00F0243490A702FD004EB82000168EC
:1003200089B2009109040CD53E4B016889B201EAFB
:10033000080101603C48197800EB810050F8040C7A
:100340008047009800060FD53648017804EB8101FC
:100350000A6892B202EA0B020A603449007801EBA3
:10036000800050F8040C8047DAF800104846A9F8DD
:1003700000100904CBD4BDE8F88F216829802988B2
:1003800001F030016980298801F4405129802168F9
:1003900089B2314081F4005181F02001394321605C
:1003A0000088C0060028206880B216DB00EA0B0037
:1003B000206000F081FC23E02988890401D580F4C5
:1003C00000506988C90624D46988890601D580F05F
:1003D000200080B238432060CDE7010507D52068B2
:1003E00080B200EA0800206000F080FF08E000040E
:1003F000BAD5206881B201EA0801216000F068FDE9
:100400002068298880B23040C904D5D580F4805056
:10041000D2E780F01000D7E716000020005C004013
:100420005600002004000020740000205800002026
:10043000074901EB80000168490408D5016848F6C6
:100440008F7289B211404CF28002114301607047F3
:10045000005C0040074901EB80000168490608D5AF
:10046000016848F68F7289B2114048F2C002114308
:1004700001607047005C0040064901EB800108689C
:1004800048F68F6280B2104048F280021043086044
:1004900070470000005C004010B5022000F0CCF86E
:1004A000002809D0022000F00DF80021034801F0D7
:1004B0002AF903490120087010BD0000002C0140FA
:1004C00033000020C10002D502490860704702498C
:1004D000486070470404024000000240002901689F
:1004E00002D041F0010102E04FF6FE7211400160BE
:1004F0007047000010B5144C204600F02BF814494A
:10050000124800220860A1F52570C1E901024FF4EC
:10051000A070C1E90302802048614000886180002A
:10052000C861202008620002C1E90902204600F0EB
:100530009BF801220221204600F08EF82046BDE8FB
:1005400010400121FFF7CABF080002404C240140BF
:10055000D803002001684FF6FE72114001600021AF
:10056000016041608160C1603149314A083990427F
:1005700003D1486840F00F0006E02D4A1432904243
:1005800004D1486840F0F00048607047284A28329B
:10059000904203D1486840F47060F5E7244A3C3249
:1005A000904203D1486840F47040EDE7204A503251
:1005B000904203D1486840F47020E5E71C4A643259
:1005C000904203D1486840F47000DDE7184A783261
:1005D000904203D1486840F07060D5E7154A111F7A
:1005E000904203D1086840F00F0006E0114A14322F
:1005F000904204D1086840F0F000086070470D4A4E
:100600002832904203D1086840F47060F5E7094A47
:100610003C32904203D1086840F47040EDE7054A4F
:1006200050329042EAD1086840F47020E5E70000BB
:10063000080002400804024001460020CA0001D51B
:10064000034A00E0034A12680A4200D001207047C2
:100650000004024000000240002A026801D00A4360
:1006600000E08A430260704730B5036847F6F072D5
:1006700093430C6A8A682243D1E904452C43224300
:100680008C692243CC6922434C6A22438C6A224300
:100690001A430260CA6842600A6882604968C160A1
:1006A00030BD00002DE9F05FDFF89C90DFF89C8002
:1006B0004FF0300AD9F8001001F11005088A0E7ABF
:1006C00008B9042E04D0AC88A04216D8042615E040
:1006D0001F490878012804D007261021A8F8001027
:1006E0002CE01C4A002012681B4B92B203EB420222
:1006F0005060A8F800A0087020E00226844200D9CB
:100700000446A0B2A968074688478346002000F047
:10071000A9FA01463A46584601F076F939460020D2
:1007200000F034FD2888001B2880688820446880F9
:10073000A8F800A009494FF440500880D9F80000FB
:100740000672BDE8F09F000008000020180000209D
:1007500000000020505C00400060004016000020B7
:100760002DE9F047234EDFF890904FF030083468C1
:1007700034F8100FA168B1B108B3A588854200D93B
:100780000546A8B20746884782462088401B20803D
:10079000608828446080002000F044FA01463A4610
:1007A000504600F0B9FB208848B114494FF440503E
:1007B00008800021084600F0E9FCA9F800802088A4
:1007C000A188884201D3032001E020B105203168CF
:1007D0000872BDE8F08731680620087208490020D9
:1007E0000968084A89B202EB41014860A9F8008013
:1007F000EFE700000800002018000020160000208D
:10080000505C0040006000402DE9F0415C4C5D4DC3
:1008100009262068002729684278062A05D0AAB14F
:10082000082A4BD00A2A4ED069E00278520666D1D7
:100830008078012804D0022804D0032804D05EE088
:10084000C96954E0096A52E0496A50E04288A2BB93
:10085000C288022A53D102797ABB0278530601D1A9
:10086000838833B102F07F02012A04D0022A0CD01F
:1008700045E045493BE08A69407900219047E0B96D
:100880002068807A0028F4D139E0417901F00F0026
:1008900001F070020B063D4951F8201003D5C1F359
:1008A0000111090102E0C1F301310903384B1B7842
:1008B000834224D90AB90029DBD120E00078400620
:1008C0001DD1344913E0027802F07F02012A16D1CB
:1008D000827AA2B1428892B9027982B9C288012A89
:1008E0000DD18A6940790021904740B92A4931B138
:1008F00020684782816100208847002006E029683F
:100900002068096940788847032808D021680A8A46
:10091000A2F57F43FF3B05D10E72BDE8F081206850
:100920000672FAE7022808D03AB10878000620D506
:10093000C888824205D9088213E04FF00800087287
:10094000EBE70ED22868154B90F82C00824201D2BA
:100950001F7006E0B2FBF0F400FB142008B9012080
:100960001870286890F82C008882BDE8F041FFF7E5
:1009700099BE032008720A4900030880CDE70000F1
:10098000080000200C000020AD140008005C0040AE
:10099000FC0000204114000885140008000000201D
:1009A00016000020704770472DE9F041DFF87CE029
:1009B0001F4F20499EF800003B7801284FF00000AF
:1009C00014D1DFF874C00022C3F10A0502EB45140C
:1009D000521C3CF81440D2B2260A0E54401CC0B23D
:1009E0000C54401CC0B24028F0D305E0FF220A544A
:1009F000401CC0B24028FAD35B1E13F0FF003870D1
:100A000005D18EF8000001210C4800F07CFE402248
:100A10000849832000F0E2FF4021032000F0B6FBEC
:100A2000BDE8F041032000F0D7BB000033000020F8
:100A3000340000205E04002044010020002C01400E
:100A400070B52F49032000F0B7FF2D490878012821
:100A500004D002280FD003283DD04BE0294C0421BC
:100A6000204600F0CFF8C0F10100C2B204212046B8
:100A700000F0D3F83EE024482149007840310128B5
:100A80004FF0000010D1214C002200BF34F812308A
:100A9000521C1D0A0D54401CC0B2D2B20B54401C53
:100AA000C0B24028F2D305E000220A54401CC0B274
:100AB0004028FAD3164909204022087010498320A3
:100AC000403100F08BFF4021032000F05FFB03204A
:100AD00000F082FB0EE04C78052C0BD20D48012271
:100AE0001146035D0C48FFF7B5FB0C480C4930F884
:100AF00014000880BDE87040032000F025BB000012
:100B00001E040020000C014033000020440100209E
:100B1000340000202E00002000240140240000208A
:100B20001A00002070B50B4C0620022520801420EE
:100B3000E070A5702146084800F012F825800020DA
:100B4000E0700320A0702146BDE87040034800F02B
:100B500007B800001C000020000C01400008014004
:100B60002DE9F041CB78002503F00F02DB0601D51B
:100B70008B781A430B884FF00F0813F0FF0F4FF0DC
:100B8000010C1CD0D0F800400E880CFA05F31E4072
:100B90009E4210D1AF0008FA07F624EA060602FAD0
:100BA00007F43443CE78282E02D0482E02D002E03B
:100BB000436100E003616D1C082DE5D304600B88E0
:100BC000FF2B1DD94468002505F108060CFA06F331
:100BD0000E881E409E420FD1AF0008FA07F624EAA5
:100BE000060602FA07F43443CE78282E00D143617A
:100BF000CE78482E00D103616D1C082DE4D34460EB
:100C0000BDE8F08102460020D2680A4200D00120EF
:100C1000704741617047016170470AB101617047D7
:100C2000416170470549096889B201EBC000044978
:100C300001EB4000806880B270470000505C0040CB
:100C4000006000400549096889B201EBC000044911
:100C500001EB4000C068C0F309007047505C0040E1
:100C6000006000400449096889B201EBC0000349F3
:100C700051F8100080B27047505C004000600040A6
:100C80000A4810B50168001D0468001D00680818B6
:100C90000BD00822064900F03DF805492046042201
:100CA000BDE81040103100F035B810BDE8F7FF1F67
:100CB000370000207047FEE710B5134C2068017A1A
:100CC000022904D0042902D0062905D015E0FFF737
:100CD000E9FC2068007A11E04178052909D1017802
:100CE000490606D1C07800F0C5F908480068006AD6
:100CF000804707480068806880470820216808729C
:100D0000BDE8104000F018B90800002010000020D5
:100D10000C000020F0B500230A2530274FF0370CD7
:100D20001C460FE0B5EB107F02D907EB107601E00F
:100D30000CEB107601F8136001EB430600015B1C1D
:100D40007470DBB29342EDD3F0BDFEE7704770479D
:100D500070B50B4C0B200026207066700125A57025
:100D6000E570204600F00EF81B202070667002200F
:100D7000A070E5702046BDE8704000F003B80000A8
:100D80002000002070B50F21C478027801234FF0B5
:100D9000E026DCB1124C246804F4E064C4F5E0649D
:100DA000250AC5F10404E9404578A54084780C4043
:100DB0002C4321010B4C1155007800F01F018B4092
:100DC000400906EB8000C0F8003170BD02F01F0042
:100DD0008340500906EB8000C0F8803170BD0000F0
:100DE0000CED00E000E400E002490843024908601D
:100DF000704700000000FA050CED00E070B52F4DC3
:100E00002868017844784A0606D001F07F0001285E
:100E100028D002282BD035E0092C06D0052C07D08D
:100E2000032C0ED0012C14D02CE000F087FB28E01E
:100E3000C1787F292ED8817861BB818851BB807AA7
:100E400027E0C17801291DD18088D8B900F092FB34
:100E500017E0C178012915D1818899B9407A8006B7
:100E60000AD40FE00B2C0DD100F0D8FB09E0012CC7
:100E700002D0032C03D005E000F06CFA01E000F092
:100E80008BFB58B10E4800684169E0B288470328DF
:100E900002D018B108200DE009200BE0094A062015
:100EA00000211268084B92B203EB42025160074ADC
:100EB000302111802968087270BD000008000020F0
:100EC0000C000020505C0040006000401800002032
:100ED00010B50F4C2068007A022811D004280FD0DA
:100EE000032804D0052802D0072805D008E0FFF722
:100EF00037FC2068007A04E006480068C068804734
:100F0000082021680872BDE8104000F015B8000004
:100F1000080000200C000020054B521C520803EB77
:100F2000410104D008C920F8023B521EFAD1704793
:100F300000600040704700000C4810B590F82C107D
:100F4000002000F0C9F80A480068007A082802D09A
:100F5000092809D006E007494FF480500880064967
:100F600010200880002010BD012010BDAC00002022
:100F700008000020160000201800002010B50120F5
:100F800000F0A4FC0648012101600021054A01602F
:100F9000031D19604FF4E05111800160002010BD65
:100FA000405C004014000020034A516821F4404195
:100FB000014351607047000000100240044A0029BC
:100FC000516901D0014300E0814351617047000045
:100FD00000100240044A0029D16901D0014300E019
:100FE0008143D1617047000000100240044A00298B
:100FF000916901D0014300E0814391617047000095
:101000000010024010B501214802FFF7EFFF012157
:101010000846FFF7D3FF01210C20FFF7E7FF01216E
:10102000BDE81040C802FFF7E1BF000001490860B9
:1010300070470000D800424207480068052809D1DF
:1010400006480168491C0160062903D1002101609E
:10105000FFF730BE70470000240100205000002040
:1010600070470000024920F0070008607047000048
:10107000505C0040F0B50E490E4E48F68F770B7865
:10108000002148F2800C0AE0CCB206EB84052A6805
:1010900092B23A40224342EA0C022A60491C994229
:1010A000F2D3044940F080004C310860F0BD0000EC
:1010B000FC000020005C0040054A21F0010112689C
:1010C00092B202EBC000034A02EB4000816070471D
:1010D000505C0040006000400D4A12683E2992B208
:1010E00002EBC0000B4A02EB400209D94809C906CD
:1010F00001D1401E80B24FF4004141EA802005E05A
:101100004808C90701D0401C80B2800210607047B7
:10111000505C00400C6000400A4A02EB80021068FC
:101120004BF68F7380B200EA0300CB0401D580F444
:101130008050890401D580F4005048F280010843B2
:1011400010607047005C0040074901EB80010868AF
:101150004BF68F7280B2104080F4405048F280020B
:101160001043086070470000005C0040054A21F011
:101170000101126892B202EBC000034A42F810105B
:1011800070470000505C004000600040044A126854
:1011900092B202EBC000034A02EB4000416070478C
:1011A000505C0040006000400A4A02EB8002106878
:1011B00048F6BF7380B200EA0300CB0601D580F089
:1011C0001000890601D580F0200048F28001084314
:1011D00010607047005C0040074901EB800108681F
:1011E00048F6BF7280B2104080F0300048F28002B2
:1011F0001043086070470000005C0040054A02EBA5
:101200008000026848F68F1392B21A400A430260C7
:1012100070470000005C004022480021026842F450
:10122000803202604FF4A063026801F1010112F400
:10123000003F01D19942F7D10168890330D51A499D
:101240000A6842F010020A600A6822F003020A608B
:101250000A6842F002020A604168416041684160E8
:10126000416841F480614160416821F47C11416032
:10127000416841F4E8114160016841F0807101600A
:1012800001688901FCD5416821F003014160416892
:1012900041F0020141604168C1F381010229FAD1A4
:1012A00070470000001002400020024008B50121F4
:1012B0000420FFF79BFE0120ADF8000003208DF80D
:1012C000020014208DF8030069460248FFF748FC2D
:1012D00008BD00000008014010B50020FFF7A6FE81
:1012E0000121BDE81040C805FFF774BE70B516486F
:1012F0000068174D81B2154800EB4101896889B239
:1013000000EB41042868017A09290FD02178017087
:1013100061784170A088FEF7E2FF29684880208943
:10132000FEF7DDFF29688880A089C8802868012130
:101330000172C08828B1FFF767FABDE87040FFF777
:10134000FBBDFFF75BFDF8E7505C0040006000402C
:10135000080000202DE9F04134480168087810F0B9
:101360007F0002D0022805D05EE0487A00F0DF005E
:10137000487247E04888002856D10879002853D1A0
:101380004A792C4C22F080001506294B54F8205045
:1013900003D5C5F301152D0102E0C5F301352D0379
:1013A0001E78034686423FD97DB3897A69B3110618
:1013B0000ED554F82010C1F3011101291ED1D8B265
:1013C0000446FFF747F830212046FFF7EDFE15E011
:1013D00004EB80052968C1F3013101290ED14BF6D8
:1013E0008F7648F2800788B1D8B2FFF721F82868D5
:1013F00080B2304080F44050384328600E48006886
:10140000406980470020BDE8F0810DE00B4890F86E
:101410002C100020FFF760FE206880B2304080F47E
:10142000405038432060E9E70220ECE70800002044
:10143000FC000020005C004010000020AC000020F8
:1014400010B5074C30B10748006800688047206835
:101450000A3010BD216801200882002010BD000064
:101460000800002010000020054A13685A8A10B1B5
:101470000868104470478888801A188200207047D6
:101480000800002010B5074C30B10748006880689C
:10149000804720680C3010BD2168012008820020A0
:1014A00010BD000008000020100000201F4910B5EA
:1014B000096860B11E48002202800A7853060AD0EB
:1014C00002F07F02012A16D0022A16D001E0022083
:1014D0000882002010BD497A8A06027802D542F0BF
:1014E000020201E002F0FD0249060270D1B210D4FE
:1014F00001F0FE010FE00E4810BD4A7902F00F0125
:1015000013060C4A52F8211007D5C1F3011106E069
:10151000017841F00101017003E0C1F301310129BB
:10152000F6D00548006800698047E4E7080000201D
:1015300002000020005C0040100000200A4810B5A6
:1015400000680A4AC1785278914203D882780AB971
:1015500082880AB1022010BD817205480068406887
:101560008047002010BD000008000020FC00002083
:1015700010000020064810B50068417A41F02001B3
:10158000417204480068C0698047002010BD000017
:10159000080000201000002070B51C4803681C489B
:1015A000597921F0800500EB85000C06046821F0D4
:1015B000800203D5C4F30114240102E0C4F3013412
:1015C0002403144D2D78954211D95A887AB974B1F3
:1015D0009A7A62B109060029016848F2800289B24C
:1015E00007DA48F6BF73194081F0100106E00220C7
:1015F00070BD4BF68F73194081F480511143016027
:101600000548006880698047002070BD0800002000
:10161000005C0040FC0000201000002010B50E4CC3
:101620000E4A20681268C178926940799047216813
:101630008A7A22B118B9087908B9887808B10220E5
:1016400010BD07480068C068804720684179C172B2
:10165000C1780173002010BD080000200C0000209C
:1016600010000020704700000F4810B5016841F0DD
:101670000101016041680D4A1140416001680C4A56
:1016800011400160016821F480210160416821F46A
:10169000FE0141604FF41F018160FFF7BDFD054968
:1016A0004FF00060086010BD001002400000FFF81D
:1016B000FFFFF6FE08ED00E010B50E4C02212046BB
:1016C00000F05AF8002813D00221204600F018F844
:1016D00001210948FEF782FD204600F04BF807493A
:1016E0000988084481B22046BDE8104000F09EB849
:1016F00010BD0000002C0140002401401A00002011
:10170000C943018270470029018802D041F00101DC
:1017100001E021F0010101807047000070B512481E
:101720004FF6FF71002481800480C4800F4D4480F7
:101730000146284600F07CF80B49103901200C8046
:1017400048800B480088C8800C81284600F028F8A3
:101750000021284600F064F82846BDE870400122C8
:10176000022100F014B8000014040020002C0140F5
:101770001A000020808E7047038A002280890B4265
:1017800000EA010001D000B1012210467047002A92
:10179000828901D00A4300E08A43828170470000B9
:1017A00030B5028C22F001020284028C8388048B03
:1017B00022F0020224F073050C882C430D89154396
:1017C0004A882A43114DA8420BD0114DA84208D097
:1017D000104DA84205D0104DA84202D00F4DA8428E
:1017E0000DD122F008054A8923F440732A4322F0E0
:1017F00004058A882A438D891D43CB892B43838026
:101800000483C9888186028430BD0000002C014019
:1018100000340140004001400044014000480140C4
:10182000028B22F008020A430283704781867047C8
:1018300030B502881B4B1C4C98420DD0A0420BD0F7
:10184000B0F1804F08D0194DA84205D0184DA842DC
:1018500002D0184DA84203D122F070054A882A43CD
:10186000154DA84206D0154DA84203D022F440756C
:10187000CA882A4302808A8882850A88028598421B
:101880000AD0A04208D00E4A904205D00D4A90429C
:1018900002D00D4A904201D1097A0186012181824C
:1018A00030BD0000002C0140003401400004004025
:1018B00000080040000C00400010004000140040F0
:1018C000004001400044014000480140044A002813
:1018D0004FF00101104601D0FFF79BB9FFF79BB90C
:1018E0000008014006480549022201600A72064AC2
:1018F0000449C0E9011208680047000028010020DF
:1019000008000020AC0000200001002008B54FF4C2
:10191000C060FFF769FA14208DF8000001208DF8EF
:10192000010000218DF802108DF803006846FFF7D2
:1019300029FA08BD70B5134D2868134C6080608883
:10194000124E31880840800507D54FF6FF502860B9
:101950002078401C2070FFF76FFB608831880840BA
:10196000000401D5FEF7C0FC6088318808404005BE
:1019700007D54FF6FF30286005484068BDE8704045
:10198000004770BD445C004054000020140000205B
:10199000AC000020FFF7CEBF0549002008600549D4
:1019A0004FF4064008800249091F08600020704774
:1019B000445C00401400002070B500F07F060D4626
:1019C0003046FFF73FF904463046FFF72BF9014652
:1019D00022462846FFF7A0FA204670BD70B500F0F9
:1019E0007F040D4616462046FFF73CF90146B2B289
:1019F0001646284600F008F831462046FFF7C6FB99
:101A0000002070BDFEE70000084B10B5521C5208C4
:101A100003EB410108D003784478801C43EA042397
:101A200021F8043B521EF6D110BD000000600040BA
:101A3000114910B50A68212802D0202807D018E0E3
:101A4000107800F07F00212813D10C490AE01078AB
:101A5000202300F07F010A48212901D0037008E00B
:101A60000849037029B10020916150828847002005
:101A700010BD022010BD000008000020A11A0008BF
:101A800090000020391C00080149FFF7EDBC000060
:101A9000A40000200149FFF7E7BC00009C000020E3
:101AA00008B10448704704490820096808820020EA
:101AB00070470000940000200800002005490968D4
:101AC000C978042901D900207047034A02EBC101FB
:101AD000FFF7CABC08000020DC00002009B901287B
:101AE00001D90220704700207047000007490968AB
:101AF000097801F07F01212903D1022803D022288F
:101B000001D002207047002070470000080000202C
:101B10003C4810B500683C4A00218172D27942727B
:101B2000C1720846FFF79EFA4FF400710020FFF7DC
:101B300065FB10210020FFF737FB40210020FFF755
:101B4000BBFA80210020FFF711FB0020FEF794FC78
:101B50002E4890F82C100020FFF7BEFA0020FFF767
:101B6000F3FA00210120FFF749FBC0210120FFF714
:101B7000FDFA20210120FFF717FB00210120FFF7CC
:101B8000CBFA4FF4C0610220FFF738FB4FF48071AD
:101B90000220FFF7EBFA00210220FFF7BDFA202117
:101BA0000220FFF701FB00210320FFF727FB4FF482
:101BB00088710320FFF780FA40210320FFF78CFA99
:101BC0004FF440510320FFF7A7FA00210320FFF74D
:101BD000EBFA00210320FFF711FB4FF4A87103205B
:101BE000FFF7C4FA40210320FFF7D0FA3021032089
:101BF000FFF7DAFA0020FFF73DFA054901200860F7
:101C000010BD000008000020FA1C0008AC000020F5
:101C1000240100200348807A002802D002490520D0
:101C20000860704728010020240100200149042099
:101C3000086070472401002008B104487047044937
:101C400008200968088200207047000094000020E6
:101C50000800002003480178202901D100210170EB
:101C600070470000900000207047000010B5FFF79B
:101C700007F80548002400688472FFF77FF9FFF732
:101C80008BFE0248046010BD0800002024010020E3
:101C900002E008C8121F08C1002AFAD17047704735
:101CA000002001E001C1121F002AFBD17047000093
:101CB000FFF7FCFAFFF710FBFFF728FEFFF712FE15
:101CC000FFF7A0F9FFF744F8FEF72CFFFFF726FD1A
:101CD000FEF710FCFEF742FA01210248FFF713FD60
:101CE000FEE70000002C014012010002020000404B
:101CF0008304405700020102030109024A00020165
:101D000000C0320904000001020201000524001095
:101D10000105240100010424020205240600010734
:101D20000582030800FF09040100020A0000000701
:101D300005030240000007058302400000070581FB
:101D400002400000040309042603530054004D0020
:101D50006900630072006F0065006C00650063003D
:101D6000740072006F006E0069006300730032033C
:101D7000530054004D00330032002000560069002B
:101D800072007400750061006C00200043004F0079
:101D90004D00200050006F007200740020002000F1
:101DA000C01D00080000002028010000901C000851
:101DB000E81E00082801002078070000A01C000889
:101DC0000000000000000000000000000000000013
:101DD000000000000000000000009411000000005E
:101DE000000000009411CA086504C201E100050367
:101DF000020000000A1A03530054004D0033003261
:101E00000031003000000000000000000000000071
:101E10000000000000000000A70900084F0D0008A6
:101E2000A90900084F0D00084F0D00084F0D0008CC
:101E30004F0D00084F0D00084F0D0008410A000823
:101E40004F0D00084F0D00084F0D00084F0D000802
:101E50000000000000C2010000000800E81C0008AB
:101E600012000000FA1C00084A0000006D1C000867
:101E7000111B0008551C0008691C0008311A0008D5
:101E8000ED1A0008DD1A0008951A0008891A0008E2
:101E9000BD1A00080000000040000000441D0008BA
:101EA00004000000481D0008260000006E1D000808
:101EB00032000000350000201A000000040100007C
:101EC0004F0D0008151C00084F0D00084F0D0008AD
:101ED0004F0D00084F0D00084F0D00084F0D000872
:081EE0002D1C000800000000A9
:04000005080000ED02
:00000001FF
